:020000040000FA
:02000000522983
:08000800FE00030E8301FF005E
:100010000A08FC00831203130C1C2D28A613C20B24
:100020002728A6170530C200C30A3C304302031D2F
:100030002728C301C10A26143C304102031D27288A
:10004000C101EF0A18306F02031D2728EF013C3071
:100050008F0032088E009016101683120313181D9D
:1000600032283428981C3B2818119810181218169A
:100070000730BD2237298C1E37290D301A0203198B
:100080009A2861301A020319D22863301A02031920
:10009000E42867301A020319C52847301A020319E9
:1000A000DE2868301A020319C32869301A020319BE
:1000B000E7286D301A020319D82870301A02031984
:1000C000CF2873301A020319E12874301A02031979
:1000D000CA2875301A020319DB2876301A02031970
:1000E000D52830301A0203191A2931301A0203199F
:1000F0001A2932301A0203191A2933301A02031945
:100100001A2934301A0203191A2935301A02031930
:100110001A2936301A0203191A2937301A0203191C
:100120001A2938301A0203191A2939301A02031908
:100130001A29372900303A020319372901303802C9
:100140000319EF28043038020319EA280530380271
:100150000319F428083038020319F9280930380245
:100160000319FC280C30380203191529063038020F
:1001700003190B2907303802031910290A303802F5
:100180000319FF283729542333290B30B8000730CF
:10019000E10033290230B8000830E100332904308F
:1001A000B8002E290130B8002E290530B8002E29BC
:1001B0000830B8002E290930B8002E290A30B800BE
:1001C0002E290630B8002E290730B8002E290C3011
:1001D000B8002E293C08BF000230E1002B293C0862
:1001E000C0000130E1002B293C08C0000330E100D1
:1001F0002B293C08C1002B293C08EF002B293C0887
:10020000B2001F242B293C08B4001F242B293C08D2
:10021000B3001F242B293C08B6000430E1002B2931
:100220003C08B6000530E1002B293C08B600093037
:10023000E1002B2930301A02B9003C08BC07BC078A
:10024000BC07BC07BC07BC07BC07BC07BC07390818
:10025000BC07BA0A372983120313B70183120313A9
:10026000BC01BA01372983120313B701B801831205
:1002700003138B138B120B128B110B118B100B10A2
:100280000C138C120C128C110C118C100C108D1381
:100290000D138D120D127C088A007F0E8300FE0E56
:1002A0007E0E0900831603130F178F160F168F117A
:1002B0000F10831203138312031385018601870134
:1002C00083120313860183160313003086008316FE
:1002D000031319309900831603139B11831603131C
:1002E0001815181283120313981783160313981600
:1002F000831203131816831203130530C200C301BF
:10030000C101EF0125268316031320309F008316B9
:1003100003133F30850083160313083086008316CD
:100320000313CA308700831203171E149E141E1570
:100330009E151E129E161E139E17831203171F145E
:100340009F141F119F11831203139F019F171F13E7
:100350009F121F169F111F151F14831603130130C0
:100360008100831603138C018C160C14831603135F
:100370000D12831203130616061786178312031332
:10038000071407150716A601831603130130810011
:10039000831203139013101390161016901110115E
:1003A000901010140030831203138F008312031374
:1003B0008E00831203130C10831203138312031392
:1003C0008B010B178B178312031332238312031332
:1003D0002F24831203138312031308306102031DB9
:1003E000F6291E26831203132D23912A8312031349
:1003F00002306102031D012A3F0883120313950096
:10040000912A8312031301306102031D0F2A9522E2
:1004100083120313F925831203132D23912A8312C8
:10042000031303306102031D222A95228312031352
:10043000032683120313EB25831203132D23831248
:100440000313912A8312031304306102031D462A09
:100450003608003A031D2E2A0616912A3608013A5C
:10046000031D342A0617912A3608023A031D3A2A38
:100470000714912A3608033A031D402A0715912ACA
:100480003608043A031D912A0716912A8312031392
:1004900005306102031D6A2A3608003A031D522AFC
:1004A0000612912A3608013A031D582A0613912A8A
:1004B0003608023A031D5E2A0710912A3608033ACD
:1004C000031D642A0711912A3608043A031D912A54
:1004D0000712912A8312031309306102031D862A31
:1004E0003608003A031D792A05080839031D822AB7
:1004F000802A013A031D912A05082039031D822A0A
:100500003030832A3130BD222D23912A83120313E8
:1005100007306102031DEB295A24831203132D2394
:10052000912A83120313E101EB298312031340087C
:100530000F39BB000310BB0D0310BB0D3B0883122A
:1005400003139F019F009F171F131F14FF30A1006B
:10055000A10BA82A9F149F18AB2A831203131E080D
:1005600083120313E200831603131E08831203137E
:10057000E300080083120313303E99008312031333
:10058000FF30A500A50BC52AC72A981CC22A8312D2
:10059000031308002615A700A8016430A702031C56
:1005A000D32AA80ACD2A003028020319DA2A2611F4
:1005B0002808BA226430A707A8010A30A702031C42
:1005C000E32AA80ADD2A00302802031DE92A261999
:1005D000EB2A2808BA220A30A7072708BA220800FF
:1005E000FD2226152E081B232F081B2330081B2352
:1005F000261D08000030BA22080003101030B10098
:10060000AE01AF01B0012E3084000330A8003330BA
:1006100080078019F039801B0F398002840AA80BEB
:10062000072BAD0DAC0DB00DAF0DAE0DB10B032B07
:100630000030AE000800AB002B0E0F39031D222B3B
:100640002619242B2611BA222B080F39031D2A2B19
:10065000261908002611BA2208000D30BD220A30E2
:10066000BD2208005030BD226130BD226E30BD2257
:100670007430BD226530BD226C30BD227430BD2285
:100680006A30BD226530BD222030BD224930BD22F6
:100690004F30BD222D30BD223030BD222E30BD2244
:1006A0003130BD222D2308004630BD226F30BD22DF
:1006B0007230BD222030BD226830BD226530BD229F
:1006C0006C30BD227030BD222030BD227330BD227F
:1006D0006530BD226530BD222030BD225230BD22A2
:1006E0004530BD224130BD224430BD224D30BD22B7
:1006F0004530BD222D230800831203138B13831270
:10070000031771088D0072088C00831603178C1371
:100710000C158B138B1B892B55308D00AA308D0047
:100720008C148B17831603178C18922B0C118312C1
:1007300003139B230800112483120313A6127208CB
:10074000831203170C02031DA82B83120313080046
:10075000AD2383120313A61608008312031365301A
:10076000BD226530BD227030BD227230BD226F3097
:10077000BD226D30BD222030BD227730BD227230C7
:10078000BD226930BD227430BD226530BD222030CB
:10079000BD227230BD226530BD227330BD2275305E
:1007A000BD226C30BD227430BD222030BD226130AC
:1007B000BD226430BD226430BD227230BD2265305E
:1007C000BD227330BD227330BD223D30BD22710881
:1007D000CA222030BD226F30BD227230BD22693066
:1007E000BD226730BD226930BD226E30BD2261302E
:1007F000BD226C30BD223D30BD227208CA2220309D
:10080000BD227230BD226530BD226130BD22643010
:10081000BD223D30BD22112483120313CA222D2391
:100820000800831203137108831203178D008316C7
:1008300003178C130C14831203170C08080083127F
:1008400003130030F1003208F2007C2383120313FB
:10085000F10A3F08F2007C2383120313080083127D
:100860000313FF30F1001124831203137B3A0319A1
:100870004A2C83120313AF30B2008030BF001F2414
:10088000831203137B30F200FF30F1007C238312CC
:1008900003130800831203130030F10011248312A4
:1008A0000313B200F10A112483120313BF00831251
:1008B00003130800831203133208CA222D230800F1
:1008C000F309F30A0319F403F4090034F309F30AF2
:1008D0000319F403F4097308F5070318F60A7408FA
:1008E000F60700341030AB007608FA007508F900FE
:1008F000F601F50100347224F801F7010310F90D37
:10090000FA0DF70DF80D74087802031D892C730891
:100910007702031C922C7308F702031CF803740877
:10092000F8020314F50DF60D0310F90DFA0DF70D8D
:10093000F80D74087802031D9F2C73087702031CBE
:10094000A82C7308F702031CF8037408F8020314B8
:10095000F50DF60D0310F90DFA0DF70DF80D7408ED
:100960007802031DB52C73087702031CBE2C730894
:10097000F702031CF8037408F8020314F50DF60DD2
:100980000310F90DFA0DF70DF80D74087802031D28
:10099000CB2C73087702031CD42C7308F702031CBA
:1009A000F8037408F8020314F50DF60D0310F90DA1
:1009B000FA0DF70DF80D74087802031DE12C730889
:1009C0007702031CEA2C7308F702031CF80374086F
:1009D000F8020314F50DF60D0310F90DFA0DF70DDD
:1009E000F80D74087802031DF72C73087702031CB6
:1009F000002D7308F702031CF8037408F8020314AF
:100A0000F50DF60D0310F90DFA0DF70DF80D74083C
:100A10007802031D0D2D73087702031C162D730831
:100A2000F702031CF8037408F8020314F50DF60D21
:100A30000310F90DFA0DF70DF80D74087802031D77
:100A4000232D73087702031C2C2D7308F702031C57
:100A5000F8037408F8020314F50DF60D0310F90DF0
:100A6000FA0DF70DF80D74087802031D392D73087F
:100A70007702031C422D7308F702031CF803740865
:100A8000F8020314F50DF60D0310F90DFA0DF70D2C
:100A9000F80D74087802031D4F2D73087702031CAC
:100AA000582D7308F702031CF8037408F8020314A6
:100AB000F50DF60D0310F90DFA0DF70DF80D74088C
:100AC0007802031D652D73087702031C6E2D7308D1
:100AD000F702031CF8037408F8020314F50DF60D71
:100AE0000310F90DFA0DF70DF80D74087802031DC7
:100AF0007B2D73087702031C842D7308F702031CF7
:100B0000F8037408F8020314F50DF60D0310F90D3F
:100B1000FA0DF70DF80D74087802031D912D730876
:100B20007702031C9A2D7308F702031CF80374085C
:100B3000F8020314F50DF60D0310F90DFA0DF70D7B
:100B4000F80D74087802031DA72D73087702031CA3
:100B5000B02D7308F702031CF8037408F80203149D
:100B6000F50DF60D0310F90DFA0DF70DF80D7408DB
:100B70007802031DBD2D73087702031CC62D730870
:100B8000F702031CF8037408F8020314F50DF60DC0
:100B90000310F90DFA0DF70DF80D74087802031D16
:100BA000D32D73087702031CDC2D7308F702031C96
:100BB000F8037408F8020314F50DF60D00347224DE
:100BC000FA0CF90C03186B24F60CF50CF80CF70C66
:100BD000AB0BE02D0034831203136A08AC006B08E2
:100BE000AD00F022831203136D30BD225630BD22BA
:100BF0000800831203136208AC006308AD00F02202
:100C00008312031308001330F400C430F3006208A9
:100C1000F6006308F500DF257508F6007808F50092
:100C20000030F4000430F3007B24831203137608B1
:100C3000AC00EA007508AD00EB0008006F08CA229E
:100C40003A30BD224108CA220800831203139101E1
:100C50008316031365309200831203133230BF00F2
:100C60008312031395000C30831203139700831231
:100C7000031392011210921012158312031308002D
:02400E00D430AC
:00000001FF
